:030000000219FDE5
:03000B000200A848
:03002B0002015A75
:03005B000202EBB3
:030073000202D8AE
:1000800002030406080C10182030406080040608A3
:100090000C10182030406080A0C00003070F1F051F
:1000A000050D050305030302C2AFC0D0C0E0206206
:1000B00014E5256009E473E525F4F58AD262D0E001
:1000C000D0D0D2AF3285268AC262E526F4602F30C6
:1000D000682520720DD0E0D0D0C292C290C291D2D9
:1000E000AF32C292C290C291206F0C206509740A8F
:1000F000D5E0FDE57B4290D0E0D0D0D2AF32758A1A
:1001000000C28DD26201F701B7306805206502D2C6
:100110009201B7306805206502D29101B7306805B9
:10012000206502D29001B7C29530680A2065077435
:1001300008D5E0FDD29201B7C29430680A20650765
:100140007408D5E0FDD29101B7C29330680A2065EA
:10015000077408D5E0FDD29001B7C2AFC2AD53E637
:10016000EFC0D0C0E0D2D3D2AFC2CEE52A60072024
:10017000744F152A21C17800790020742EE5803053
:100180007E01F430E70278FF53DACF207E0343DAB2
:1001900020307E0343DA10C2D8C271E580307E0180
:1001A000F430E70279FFC3E89970CB306103752A18
:1001B00018207403752A18885CD270E86003755F94
:1001C0000020740DE52B6004152B21D143DA01C208
:1001D000D82070024144A85C206102C270207431B2
:1001E000C3E894F0400374F0F8E8C4540F28F87999
:1001F00084B703024111C313C3138721200802C32C
:1002000013200A06C3C898F8411128F8500374FF58
:10021000F8C3E895655003E565F88822E52D540696
:100220006022206B1FE536C333C333F8E564C31384
:10023000C313F9C3952240028922E82522F52250F2
:10024000037522FF852224A824C3E524956140027A
:10025000A8618825E56670024188C3E8AA669A50BD
:1002600003E8FAE4F9EAC333FBE568F45B29400DDF
:100270002567F8E56760021567400B41880AC3E50A
:10028000679A5002056778FF8826C26FC3E52694F7
:10029000F84002D26F20CF0AD0E0D0D043E610D28F
:1002A000AD32C2CF053A7801E52A600530740215F7
:1002B0002AC3E55C94014005755F0041CE7560007E
:1002C000756900E55F2401F55F5003755FFFD0E0BD
:1002D000D0D043E610D2AD32C2AF53E67F7592FA6A
:1002E0007593FFC260759104D2AF32C2AF53E6EF8F
:1002F000C2ADC0D0C0E0C0F0D2D3D2AFA8FBA9FC41
:10030000C2D8307102615253DACF207E0343DA1033
:10031000307E0343DA20D271E580307E01F420E79D
:1003200002612988278928A17F53DACF207E0343E1
:10033000DA20307E0343DA10C2D8C271307402A1D1
:100340006B7800E580307E01F430E702A16B885CB9
:10035000A15353DACF207E0343DA20307E0343DA01
:1003600010C271206102812B53DACF207E0343DA61
:1003700010307E0343DA20C2D8D27188578958C31F
:10038000E89555F8E99556F97B007E087A00C3E8B0
:10039000948CE994005005755B00811D882178A23A
:1003A000E6A8216055C3E894C8E994005008E4D257
:1003B000E4FB7A0A61F8C3E89468E994015008E420
:1003C000D2E3FB7A0F61F8C3E894D0E994025008B5
:1003D000E4D2E2FB7A1E61F8C3E894A0E9940550E8
:1003E00008E4D2E1FB7A3C61F8C3E89498E9940808
:1003F0005008E4D2E0FB7A787E00C3E89559FCE926
:10040000955AFD30E70AECF42401FCEDF43400FDCC
:10041000755B00C3EC9AED9E5003755B01885989AA
:100420005A8557558558567802A153C3E89527F841
:10043000E99528F9307C02A137307B02A137307A68
:1004400002A130207502814EE9FDE8FC816DE9C30F
:1004500013F9E813F8307902A130E9C313F9E8136E
:10046000F8307802A130E9C313FDE813FC20612CB9
:0F047000C3EC941CED940240028184ED701EC316
:10047F00EC94C850180529E52970021529C3E52900
:10048F00940A5002A16B755C00D270A16BE52960D4
:10049F000215297888E6F97400207F087896B90349
:1004AF0002789EE624FAFEE43400FFC3EC9EFCEDD6
:1004BF009FFD9208B90310A2085007207609D27643
:1004CF0081D6307602C276A2085016B9030DECF42D
:1004DF002401FCEDF43400FD0204F078007900A152
:1004EF0037B90315EC33FCED33FDC3EC940AFCED87
:1004FF009400FD50047C007D00C3EC94FFED94004C
:10050F00400678FF7900A137EC8572F0A4C5F0A200
:10051F00F733F87900400302055378FF790002059D
:10052F0053E9C313F9E813F8307C0EE9600278FF42
:10053F00C3E81338F8E43400F9C3E894FFE99400F2
:10054F00400278FF885CD270206102A16B741FF4A7
:10055F00552F4BF52FC274EB7002D274752A1830D9
:10056F007403752A0A306102A17F20740353DAFEE7
:10057F00207403752B06D0F0D0E0D0D0D2AD43E677
:10058F00103279010205AF79030205AF790A02052E
:10059F00AF791E0205AF79640205AF79C80205AFC6
:1005AF007817E4D5E0FDD8FAD9F6227A147B7802D1
:1005BF0005D67A107B8C0205D67A0D7BB40205D650
:1005CF007A0B7BC80205D6E573D5E001227902E4E8
:1005DF00C294D5E0FDD291D5E0FDC291D5E0FDD218
:1005EF0094D5E0FDE920E002D29230E002D290E50E
:1005FF0073D5E0FDE920E002C29230E002C29074B0
:10060F0096D5E0FDD9C9EAF8D5E0FDD8FBDBB8C235
:10061F009422C37C007D0075F00005F0EA33FAEBFD
:10062F0033FB50F6EB13FBEA13FAC3E9FFE8FEE8DE
:10063F009AF8E99BF95004EFF9EEF8B3EC33FCEDBF
:10064F0033FDD5F0DFEDF9ECF822E889F08A20D2FE
:10065F00D4F8A9F07B0030F70B7BFFF42401F8E905
:10066F00F43400F9E88520F0A4ADF0F8E98520F026
:10067F00A4AFF0FEED2EF974003FFA7C04C3EA1329
:10068F00FAE913F9E813F8DCF48BF030F70AE8F421
:10069F002401F8E9F43400F9E889F0C2D4F8A9F09C
:1006AF002222C3E54113F9E54013F8C3E54498F856
:1006BF00E54599F9500CC3E89480E994FF40160280
:1006CF0006E8C3E8947FE9940050030206E8787FB8
:1006DF0079000206E8788079FF8849894A22E5493E
:1006EF002546F8E54A3547F9854A20E4300701F4F5
:1006FF003548FA30E709C3EA94F04015020726C3DC
:10070F00EA940F500302072678FF79FF7A0F02074A
:10071F0026780079007AF0C3E5249561500AC374F6
:10072F00019524500B020744E54A20E70E020744C7
:10073F00E54A30E706884689478A482278A5E6FACF
:10074F00C3E54933F8E54A33F9D159E930E70BC32B
:10075F00E89480E994FF4013E17EC3E8947FE99425
:10076F00005002E17E787F7900E17E788079FFE8A2
:10077F0020E715C3E52398F84009C3E89401400327
:10078F000207A578010207A5E8F424012523F84004
:10079F00030207A578FF884B2278A6E6FAA847A997
:1007AF0048D159E930E70CC3E89401E994FF4016AA
:1007BF000207D9C3E894FFE9940050030207D978E0
:1007CF00FF79000207D9780179FFE920E715C3E522
:1007DF004B98F84009C3E8940140030208007801E0
:1007EF00020800E8F42401254BF8400302080078C2
:1007FF00FF88242278FF20692879A1E76023E5414B
:10080F00601F74FF8541F0848539F0306A0375F0FD
:10081F0005A4F8C5F0600278FFC3E895645002A8FC
:10082F0064886322C3E5409440E5419401E5635039
:10083F0003140144046002F5632202084C2275E898
:10084F0090227883E6FF30EDF9A8BDA9BE0570C3ED
:10085F00E57094084052757000E9FA79A0E760449A
:0E086F00EA7007E571601B020885C3E8957109
:10087D006010E5715006600C140208910460F902D5
:10088D000891E571F571C3946D401B7561C0C394FA
:10089D00044013756180C39404400B756140C3948B
:1008AD0004400375610075BB0622E561F460020525
:1008BD0061E570B4070375BB1022743279A787F018
:1008CD00A4C5F0A2F733F8C3E895614002A861888A
:1008DD00228824882588268864227540007541F079
:1008ED0022C2AF75C820A8CCA9CDAA3A30CF010A33
:1008FD0075C824D2AFAB3BAC3C883B893CC3E89B6D
:10090D00F8E99C206908F930660221FF2159AD3DB7
:10091D008A3DF9EA9DFA600678FF79FF213EAE3EE9
:10092D00AF3F8B3E8C3FA83BA93CC3E89EF8E99FA7
:10093D00F9C3E54113FBE54013FAE82AF540E93B1D
:10094D00F54150067540FF7541FF21A6AA40AB4108
:10095D00AC40AD417E047F02C3EB9404400D1E1FDD
:10096D00C3EB94084005206A021E1FC3ED13FDEC76
:10097D0013FCDEF7C3EA9CFAEB9DFBEF6009C3E9BC
:10098D0013F9E813F8DFF7EA28FAEB39FB8A408B05
:10099D004150067BFF8B408B41C3EB94025002D23A
:1009AD00663069047F0321D17892E6FFC3E5379461
:1009BD008240110FC3E53794A040010FC3EF940699
:1009CD0040027F057E02E541C4540FF9E541C45450
:1009DD00F0F8E540C4540F28F8C3E89EFAE99400F6
:1009ED00FB4009C3EA9402EB940050047A02E4FB45
:1009FD00414BAA40AB41EBC4FEEAC4540F4EFCC3BD
:100A0D00EA9CFAEB9400FBC3E813C313F8EA28FA47
:100A1D00EB3400FB8A408B41C3EB94024002C2666B
:100A2D007802EBC4FE7B00EAC4540F4EFAC3EA9879
:100A3D00FA4005C3940250027A027892E6FF3060C4
:100A4D0002414B855192855293D26043E680C3E4B7
:100A5D009AF8E49BF930660241D7E8FAE9FBD3E94D
:100A6D0013FDE813FC88518952C3EF94036038EFEE
:100A7D0020E00DE82CF8E93DF9ECFAEDFB020AA0B7
:100A8D00E828F8E939F9C3E82402F8E93400F97ADD
:100A9D00FE7BFFC3EF9403400E8A538B54884D8920
:100AAD004E8C4F8D50610B885389548A4D8B4E8CD3
:100ABD004F8D503069127553F07554FF754FF075A9
:100ACD0050FF7551F07552FF610BE8FAD3E813FC36
:100ADD008851C3EF94036020EF20E007E82CF8EC79
:100AED00FA41F7E8282402F87AFEC3EF9403400890
:100AFD008A53884D8C4F610B88538A4D8C4FE56816
:100B0D00C3335002646BF5683060026115753402B1
:100B1D00D26043E680E52D54066034A840A941C358
:100B2D00E913F9E813F8C3E913F9E813F830690488
:100B3D00E92440F9C2AF53E67F759100C3E498F5FF
:100B4D0094E499F595759104D26043E680D2AF2275
:100B5D00D264754300752000306C03752040020B84
:100B6D007CD264754300752040306C03752000788D
:100B7D00017901206620E52D54066002C2647914C6
:100B8D00E541C313700104F8C39414400278143086
:100B9D006904781B791B206010E543600C306903F4
:100BAD00D53404D26D8127711D0543E59BF4544066
:100BBD00B52002811130690908C3E8994001186117
:100BCD00A320640A08C3E8994002617C61A3C26452
:100BDD00C2AF53E67F75910030661275940075951E
:100BED00F8759104D26043E680D2AF617CE5417E19
:100BFD00FFC3334005C3334001FEC3E49E7594002B
:100C0D00F59561EEC3E53394015002617C306402C9
:100C1D00617CD802812561A3C26DC2AF53E67F7599
:100C2D009100855394855495759104854D92854E0B
:100C3D0093D26043E680D2AFE52D54066008206A5A
:100C4D00020533020C63306D0D206C0A206407150C
:100C5D0081158102152F2278003064027801E53765
:0E0C6D0075F007A4F9E5F028F5F0E9A2F01300
:100C7B00A2F113A2F213F537C394785003753778AA
:100C8B00C3E53795384008D265C292C290C2913005
:100C9B006002819A854F92855093D26043E6802201
:100CAB00207D16C2AF754202C294D295306202D239
:100CBB0090D2AF759F11020E9BC2AF754202C294C8
:100CCB00D293306202D292D2AF759F11020E9B303B
:100CDB007243207D20C2AF754203900138757B10A3
:100CEB00C290C293306204D29181F8D294D2AF7584
:100CFB009F01020E9BC2AF754203900138757B10AA
:100D0B00C292C295306204D291A118D294D2AF751F
:100D1B009F21020E9B207D17C2AF754203900113DA
:100D2B00C290306202D291D2AF759F01020E9BC26C
:100D3B00AF754203900113C292306202D291D2AFCF
:100D4B00759F21020E9B207D16C2AF754204C29582
:100D5B00D293306202D291D2AF759F21020E9BC209
:100D6B00AF754204C293D295306202D291D2AF7565
:100D7B009F01020E9B307243207D20C2AF7542054E
:100D8B00900127757B20C291C294306204D292A14C
:100D9B009ED295D2AF759F11020E9BC2AF754205C5
:100DAB00900149757B08C291C294306204D290A124
:100DBB00BED293D2AF759F11020E9B207D17C2AF8F
:100DCB00754205900109C291306202D292D2AF7581
:100DDB009F11020E9BC2AF75420590011DC291304F
:100DEB0062EBD290D2AF759F11020E9B207D16C283
:100DFB00AF754206C293D294306202D292D2AF75D3
:100E0B009F01020E9BC2AF754206C295D29430620F
:100E1B0002D290D2AF759F21020E9B307244207D7F
:100E2B0020C2AF754201900149757B08C292C295F1
:100E3B00306204D290C144D293D2AF759F21020E7F
:100E4B009BC2AF754201900127757B20C290C29364
:100E5B00306205D292020E65D295D2AF759F010218
:100E6B000E9B207D17C2AF75420190011DC29230BF
:100E7B006202D290D2AF759F21020E9BC2AF754218
:100E8B0001900109C290306202D292D2AF759F01DC
:100E9B00C26522900107757B00C292C290C291C2BB
:100EAB0095C293C294C26222788076FF0876FF08BF
:100EBB0076FF0876FF08760308760408760908762D
:100ECB0003087601087601788C76010876FF0876A0
:100EDB00FF0876FF0876FF0876FF0876030876FF93
:100EEB000876FF0876FF0876250876D00876FA088C
:100EFB0076FA0876040876FF0876010876000876FD
:100F0B007A0876FF087601087601087600087603E2
:100F1B00087600227887E6FFC272BF0302D272788E
:100F2B0088E6C394036008C27DE630E102D27DC23D
:100F3B007E7889E630E102D27EC3EF9402600875B9
:100F4B008E01D273020F57758E00C273227880E622
:100F5B00149000809378A5F67881E6149000809326
:100F6B0078A6F67886E61490008D9378A7F67886A7
:100F7B00E6F539C394025003753902789CE675384F
:100F8B00FFB402037538A0B4030375388278A3E667
:100F9B001490009A93F566D19E22227896E6FA7801
:100FAB0097E6FB7888E6B40305C3EB940EFB307F22
:100FBB00047A007BFFC3EB9AFCC3948250027C82C1
:100FCB007572000572EC8572F0A4C3E5F0947D4058
:100FDB00F222D27FF1A61205A01205A07A007B00A7
:100FEB007C10120596E55C2AFA74003BFBDCF37C63
:100FFB0004C3EB13FBEA13FADCF7FEC27F120FA656
:10100B0022757C00757D00E5EF20E6037520000559
:10101B0020903FFFE520146006901DFF14600093A5
:10102B0004600375EF1653D9BF7581C043FF80125F
:10103B00059175EF0643B203E5B3240220E70DF5E6
:10104B0021E5E320E0068521B343E301120E9E75F3
:10105B0080FF75A40075F19175D47F75900075A50F
:0D106B003F75F23F75D50075A60175E24195
:10107800120E9EE4F8F6D8FD756801120EB312152B
:101088008078988673753001C2AF1205AA1205BA26
:101098001205A01205C11205A01205C81205A0125A
:1010A80016A91205AA1205AA1205A5C2AF757C00D9
:1010B800757D0078FA79FA308707D9FBD8F7021CD2
:1010C80000120F1F120F58120FA5120FA67898863C
:1010D80073120E9E75881075890275C8247591045F
:1010E80075D84075A82275B80275E690759B80750D
:1010F8009D0075D10E75BC5875BB0675BA1175E89B
:1011080080120591D2AF12084975360053DACF2004
:101118007E0343DA20307E0343DA1043DA01C2D873
:10112800C2711205AAD2617B037A0CE55B70077A5B
:101138000CDB030210B31205A02070030210B3C227
:1011480070E55CC3940240E1E52F541F855E5DF5B0
:101158005EB55DD5DAD5C26153DACF207E0343DAB6
:1011680020307E0343DA10C2D8C27178A2E6700834
:10117800D274E52F54E0F52FC2757529001205A524
:10118800307409C3E529940A4002D275120596788D
:10119800023074027800C3E55C9840F0C2AF1205D3
:1011A800BA1205BA1205BAD2AF1205AA754C007860
:1011B80088E6B4030241B3120596788CE6C394011D
:1011C80050030212B3E530C3940150030212B37501
:1011D8007CA5757DF1207435C3E55C94FF5003024E
:1011E80012B3C2AF1205CFD2AF1205A5C3E55C9406
:1011F8000150EFC2AF1205BA12059B1205BAD2AF61
:101208001205A5C3E55C94FF40E902172E7F05D2BD
:101218007F120FA61205A5C2AFC27F120FA6AE5C41
:10122800C3E55C947FD2AF500241C3120591C2AFAF
:101238001205CFD2AFDFD8120FDDC3EE9405789731
:10124800F61205AA1216B17F0AD27F120FA612054E
:10125800A5C2AFC27F120FA6AE5CC3E55C947FD275
:10126800AF50E4120591C2AF1205BA12059B1205E0
:10127800BAD2AFDFD4120FDDEE24037896F6F879F0
:1012880097E7C394824003985006E824827897F63B
:101298001205AA1215CE1216E01205A5120FA6C342
:1012A800E55C94FF500221D702172E757C00757DEE
:1012B80000C3E55C954C4003855C4C1205A578019C
:1012C8007988E7B403027805C3E55C98400221B742
:1012D800C2AF1205CF1205CF1205CFD2AF1205AAA1
:1012E800753000E4F531F5320531E531F4703F052C
:1012F80032789AE67819146012783214600D787D85
:1013080014600878FA146003753200C3E532984017
:101318001D120E9E1205911532753100789986734B
:10132800C2AF1205CFD2AF789886731205A5120501
:101338009BE52A700530740201B3780120740278A5
:1013480006C3E55C9840A17888E6C394036003125D
:1013580005A5E52A70030210B3C2AF120E9EE4F58C
:1013680022F523F524F525F526F567D2AF7885E62D
:10137800C333F565E4F544F545F546F547F548F515
:1013880070F52CF52DF53775700875BB10120591A1
:1013980012084D30EDFDA8BDA9BEE97001F88871AD
:1013A80012085175700875BB10120F1FC2AF756116
:1013B800FF1208C7852261852262852263D2AF7534
:1013C8002201752401752501752601856069756AF4
:1013D800017888E6B40307C27D307602D27DD268F0
:1013E800D269753300120DF7120E261208E712089B
:1013F800EE1208E71208EE1208E7120B6E1206B09A
:10140800120C64120CAB1208EE120B5D306E031254
:1014180006B1206603120803306603120833120C63
:1014280064120CDA1208EE120B6E306E031206ED1F
:10143800120C64120D511208EE120B5D306E03127D
:10144800074B120C64120D801208EE120B6E306EF0
:10145800031207A8120C64120DF71208EE12084DB9
:0F146800120B5D120C64120E261208511208EEC0
:1014770030692F856461856462856069756A017961
:10148700187A0CC3E53399400CC269D26A8A35755C
:1014970061FF0214A9C3E55C940140030214020230
:1014A7001537306A25206C22E535147006C26AD2DA
:1014B7006B8102F535C3E55C9401400302140278A1
:1014C70088E6C3940360030215377536007882797E
:1014D700A4E760027803C3E55F985054307404E5CD
:1014E7002A604D7888E6B40317207D05207607A18A
:1014F70007307602A107206C07D26C8564618141B1
:1015070078F0306C058564617820C3E54198500216
:101517008102306C1BC26CC27D307602D27DD26AEA
:1015270075351285646181020536E55C6002A13A72
:10153700753600C2AF120E9E7887E6FE7602120F4E
:101547001F7887EEF6E4F522F523F524F525F52631
:10155700F565752C00752D00D2AF1205A5120E9EEC
:1015670078A4E66006D292D291D290307409C3E58E
:10157700369404400201B341EB901A0D78201216FD
:1015870010E520B45A0CA3121610E520B4A50302E7
:1015970015AE757CA5757DF1120EB31215CE757C4F
:1015A70000757D000215CD901A0378807B0A12160C
:1015B70010A308DBF9901A0F788C7B19121610A369
:1015C70008DBF9901A2822C2AF1216531216309070
:1015D7001A00740E121615A37409121615A37415A2
:1015E700121615901A0378807B0A121614A308DBCB
:1015F700F9901A0F788C7B19121614A308DBF912CD
:101607001666121644901A2822E493F622E6438FB0
:1016170001538FFDFFC3E583941C400122EF857CB6
:10162700B7857DB7F0538FFE22438F02438F018525
:101637007CB7857DB7901A0DF0538FFC22901A0D59
:10164700745AD115901A0E74A5D115227A3079D013
:101657007820901A40D110E520F709A3DAF7227A0B
:101667003079D0901A40E7D11509A3DAF922AB7483
:10167700A875BB01027984BB02027985BB03027995
:1016870086BB04027992BB05027987BB060279A360
:10169700BB0702799CBB08027988BB09027989E8F4
:1016A700F7227C051205AADCFB22C2AF1205BA128B
:1016B70005C11205C81205CF12059B1205BA1205FE
:1016C700C11205C81205CF12059B1205BA1205C132
:1016D7001205C81205CFD2AF22C2AF1205CF12052D
:1016E700C81205C11205BA12059B1205CF1205C80B
:1016F7001205C11205BA12059B1205CF1205C812B1
:1017070005C11205BAD2AF22AE74AF75C2AF1205CA
:10171700BA1205BA1205BA12059BDEF21205CF12EC
:10172700059BDFF8D2AF22D1B1D1A9D1A975740138
:10173700757501757600F10F7C05AD5C1205AAC3BE
:10174700ED955C70F5C3E55C9401400AC3E55C94D4
:10175700FF403202176AD175B1CED1B1C2AF75EF72
:1017670016D1A9DCD50576C3E5769403500280C669
:10177700D1A90575E5741490009F93F808C3E57522
:1017870098500280AED1A9D1A90574C3E574940A13
:101797005002809C120EB3B1CEC2AF75EF16D1A91D
:0319FD0002100CC9
:101A00000E0915FFFFFFFF0304090301015AA50199
:101A1000FFFFFFFFFF03FFFFFF25D0FAFA04FF01DE
:091A2000007AFF0101000300FF40
:101A40002358503335415357232020202020202075
:101A500023424C48454C4923463333302320202031
:101A60002020202020202020202020202020202076
:101C0000C2AFC2D353D9BF7581C043B20343FF8073
:101C1000752438752503B1DC7529A5752AF175E29F
:101C20004043F18053A47F75D4FFD2877DFA7803B7
:101C300079E67C10752200752300901DE97B0675FE
:101C400024987525013087028145208708D8FBD963
:101C5000F9DCF781B7308708D8FBD9F9DCF781B711
:101C6000B19CE493A3C39A6004DDC381B7DBDBB10D
:101C70008E6002812E7B08E493FAA3B16FDBF87AC1
:101C800030B16F752200752300B18EEAFCEBFDC305
:101C9000ED94FE400EB18E8A278B28ED30E0048A49
:101CA000828B83B18E7AC270D8C3ED94FE601950D6
:101CB000CEBD002BEC600F7520007521FF7529004B
:101CC000752A000200008100A827A9280809D80465
:101CD000D90281DCB192EA89AAF281CE0D81A3C337
:101CE000ED94035053EDA2E092007AC5C3E58294CF
:101CF00000E583941C508A200010438F02438F011B
:101D00008529B7852AB7F0300029A827A92808090E
:101D1000438F01538FFDD804D902A133C3E58394C7
:101D20001C4003A3A11689AAE28529B7852AB7F02A
:101D3000A3A116538FFC817F7AC1BD030CE493A34A
:101D4000FAB153DCF8B14B817F8181AA22AB23B178
:101D50006FEBFAEA6222752608C3E52313F523E543
:101D60002213F52250066323A0632201D526EAB18F
:101D7000DCB1DC75260AEAF4200102D287300102C8
:101D8000C287B1DCC3134002C201D526EB22B19257
:101D9000EAFB208702A192308702A197752608AE40
:101DA00024AF25C3EF13FFEE13FEB1E0B1DCC3EAAD
:101DB000133087024480FA30E703632201C3E5232E
:101DC00013F523E52213F52250066323A0632201B5
:101DD000D526D9E52265236523F52222AE24AF2539
:101DE0000E0FDEFEDFFCD20122424C48656C6934E6
:071DF000373164F3300601F6
:00000001FF
